:0200000480007A
:100000006F000005732F2034930F80006308FF03F7
:10001000930F90006304FF03930FB0006300FF038E
:10002000130F000063040F0067000F00732F2034CC
:1000300063540F006F00400093E19153171F0000BD
:1000400023223FFC171F000023200FFC6FF01FFF2F
:100050009300000013010000930100001302000050
:100060009302000013030000930300001304000038
:100070009304000013050000930500001306000020
:100080009306000013070000930700001308000008
:10009000930800001309000093090000130A0000F0
:1000A000930A0000130B0000930B0000130C0000D8
:1000B000930C0000130D0000930D0000130E0000C0
:1000C000930E0000130F0000930F0000732540F102
:1000D0006310050097020000938202017390523072
:1000E000735044749702000093820201739052305F
:1000F00073500018970200009382420273905230AE
:100100009B021000939252039382F2FF7390023B82
:100110009302F0017390023A73504030970200004E
:1001200093824201739052307350203073503030BC
:100130009301000097020000938202ED7390523009
:10014000130510001315F501635C05000F00F00F97
:10015000930110009308D005130500007300000000
:1001600093020000638A020073905210B7B200003D
:100170009B829210739022307350003097020000DF
:100180009382420173901234732540F17300203042
:10019000930120009307F0FF97200000938080E6F2
:1001A000038700009303F0FF631A77249301300064
:1001B00093070000972000009380C0E4038710009D
:1001C00093030000631C772293014000930700FF14
:1001D00097200000938000E303872000930300FF33
:1001E000631E7720930150009307F00097200000D2
:1001F000938040E1038730009303F0006310772081
:10020000930160009307F0FF972000009380B0DF18
:100210000387D0FF9303F0FF6312771E93017000F2
:1002200093070000972000009380F0DD0387E0FF34
:10023000930300006314771C93018000930700FF71
:1002400097200000938030DC0387F0FF930300FFCA
:100250006316771A930190009307F000972000002F
:10026000938070DA038700009303F0006318771817
:100270009301A000972000009380C0D8938000FED7
:10028000838200029303F0FF639A72169301B00019
:1002900097200000938000D79380A0FF8382700096
:1002A00093030000639C72149301C00013020000CA
:1002B00097200000938010D50387100013030700D8
:1002C000930300FF631C73121302120093022000B9
:1002D000E31052FE9301D0001302000097200000AB
:1002E000938060D2038710001300000013030700FF
:1002F0009303F000631473101302120093022000A2
:10030000E31E52FC9301E00013020000972000005E
:10031000938040CF038710001300000013000000FB
:100320001303070093030000631A730C13021200F7
:1003300093022000E31C52FC9301F0001302000022
:1003400097200000938010CC03871000930300FFD8
:100350006316770A1302120093022000E31252FE82
:100360009301000113020000972000009380A0C9B0
:1003700013000000038710009303F0006310770858
:100380001302120093022000E31052FE93011001A9
:1003900013020000972000009380C0C613000000E5
:1003A0001300000003871000930300006318770414
:1003B0001302120093022000E31E52FC930120015D
:1003C00097220000938202C40381020013012000DF
:1003D00093032000631471029301300197220000FF
:1003E000938242C203810200130000001301200027
:1003F0009303200063147100631030020F00F00FAC
:10040000638001009391110093E111009308D005DE
:1004100013850100730000000F00F00F930110001E
:100420009308D0051305000073000000731000C08E
:0C043000000000000000000000000000C0
:1010000000000000000000000000000000000000E0
:1010100000000000000000000000000000000000D0
:1010200000000000000000000000000000000000C0
:1010300000000000000000000000000000000000B0
:081040000000000000000000A8
:10200000FF00F00F000000000000000000000000D2
:040000058000000077
:00000001FF
